:1000000025C0189518951895189518952FC218950C
:10001000189528C21895189518951895189518953B
:1000200018957DEEEDEBDEDDDBBEBDBBE7D7B77728
:100030007E7B807E7A77726E67635B564D4B47445A
:10004000403C34302926201E191713000FE50DBF40
:1000500002E00EBF40E043BF00270EBD45E049BFB0
:10006000789454E660E0F4D15A95E9F754E660E0FC
:10007000EFD15A95E9F78BD185D100E109BF04EFA3
:100080000BBD04E20ABD0AE00EBD0FEF07BB11274E
:1000900030E0E0E6F0E007E400833EC13B3049F0A9
:1000A0003C3049F03E3049F0313119F0323119F02D
:1000B000F4CF00E03DC004E03BC0AA2705E508BB43
:1000C0000FE004BB00EF05BB0000000000000000D3
:1000D00003B3402F00EF04BB0FE005BB000000009E
:1000E0000000000003B3402BE2E2F0E090E0C8958E
:1000F000401529F093959A3001F33196F8CF98BBCB
:100100009D30A9F0A03031F0A13039F0A23061F07B
:1001100071F09F5FA395892FD3CFA395865F9150F0
:100120000AF0FCCF8A50CCCFAA278827C9CF2BC092
:1001300007B978940AE00EBD06B10074E9F306B180
:100140000074E9F724B185B107B10770003019F0E8
:10015000043041F1A2CF08E00EBDAA27992780E222
:10016000275020300CF420E03B3009F096CFA395C7
:100170002A500AF0F9CFA150265F922F00E3900F8A
:10018000A00FA3D08ACFE2E3F0E031968A9511F078
:100190003196FCCFC895A02DA8BBE0E6F0E0A08387
:1001A0003CE07CCF08E00EBD879527958795279585
:1001B000422F313109F475C0E2E3F0E071E0C895F7
:1001C000401534F47395793111F03196F8CF65CF3D
:1001D000A0E390E38BE27A3061F17B3061F17C3017
:1001E000D9F07D3059F17E3031F17F3051F17031ED
:1001F000B1F0713149F17231A1F0733141F17431D3
:1002000091F0753139F1763181F0773131F1783112
:1002100071F026C0A3E33FC095E3A2E33CC0A4E392
:100220003AC0A5E338C0A6E336C0A7E334C0A8E3CC
:1002300032C0A2E330C0A2E393E32DC0A2E397E370
:100240002AC0A3E395E327C0A4E395E324C0A5E374
:1002500095E321C0A6E395E31EC0A7E395E31BC089
:10026000793089F07830A9F0773081F0753071F00D
:10027000743079F0733039F07230D9F2713061F244
:10028000763049F00ACFA1E395E305C0A0E395E3FA
:1002900002C0A1E300C0763014F417D002C08DE292
:1002A00014D0E0E6F0E00080002D9250A02FA65080
:1002B000201744F42A171CF4C098C19AEECEC198B6
:1002C000C09AEBCEC098C198E8CE40E895D040E007
:1002D00043BF482FA6D0000040E043BF4A2FA1D023
:1002E000000040E043BF492F9CD00000313199F01D
:1002F000323189F03B3011F03C3019F0F4E0ECE79A
:1003000003C0F4E0E6E700C0C895002021F0402DCE
:1003100088D03196F9CF08951395183231F0143101
:1003200009F007C03F9331E1B9CE10E03F9332E1CD
:10033000B5CE313119F0323109F03F930FE004BBF3
:1003400000EF05BB000000000000000003B3402FD9
:1003500000EF04BB0FE005BB000000000000000040
:1003600003B3402BE2E2F0E030E0C895401529F0FD
:100370003395303129F03196F8CF0F913F5F8ECE13
:100380003F918CCE41E038D060E062D0089540E0EB
:1003900042BB4FEF41BB60E05BD043E042BB00009B
:1003A000949A949860E054D043E042BB0000949A41
:1003B000949860E04DD043E042BB0000949A94983A
:1003C00060E046D042E042BB0000949A949840EF2F
:1003D00041BB40E211D04CE00FD046E00DD0089573
:1003E00040EF41BB959A9698949A949800B3949A4A
:1003F000949803FDF9CF08954F93F2DF4FEF41BB7F
:100400004F914F9342954F7042BB0000949A94983D
:100410004F914F7042BB0000949A949840EF41BBBB
:1004200008954F93DDDF4FEF41BB4F914F934295BE
:100430004F7042BB969A0000949A94984F914F70D7
:1004400042BB969A0000949A949840EF41BB08955D
:100450004FB74F9362BFE89444E043BFFEF74F911C
:100460004FBF0895689440E043BF18951FB605EC50
:1004700006B91FBE18952043202000002050534984
:0204800000007A
:00000001FF
